:0E000000802EFF022700FFFFFFFFFF022429D2
:0300230002024F87
:20002E00C77B7581357508FF7509BF90AEBCE4F01249A2020030C82581C822C92581C97A85
:20004E000022D083D082CF2581F581CFC082C08322CF2581F581CF22FBE0CB22FCE0FBA34C
:20006E00E0CC22FAE0F9A3E0CA2229F9E5F03AFA22CB20E704CB7C0022CB7CFF2220E70463
:20008E0075F0002275F0FF22FDE493FF7401934F7004A3A3800C740293B50510740393B5A3
:2000AE00F00AE493C0E0740193C0E022A3A3A3A380D7FEEBA4FD8EF0ECA4FCEB8EF0A4C50E
:2000CE00F02C2DC5F02211DA8EF0ED22C002C001AAF0F97E007D007F11C3E933F9EA33FAEA
:2000EE00DF08F5F0E9D001D00222ED33FDEE33FEC3ED9BF5F0EE9C40E0ADF0FED380DBBBDE
:20010E00000122C333C5F033C5F0DBF722BB000122C3C5F013C5F013DBF722240280022436
:20012E0001C5F03400C5F022C394028003C39401C5F09400C5F022313BF4C5F0F4C5F022BC
:20014E0045F070220422319D4024801A319D401E7014801A319D400E7014800A319D500E38
:20016E00800431B16008E4F5F02231B160F8E4F5F0042231B140F780ED31B140F170E7801F
:20018E00ED31B140E170E780DD31B150E180D7C39BC5F09C20E70720D207C345F02220D281
:2001AE00F9D322C5F0C39C7003E5F09B2290AEBCE0A360EEE0FFA3E0A3CF2582F582EF3549
:2001CE0083F58380EB7E00CF2508F582EE3509F583EF227E00CF2508F9EE3509FAEF227EDD
:2001EE0000C5082FC508C5093EC50922E4F50AA88108E4F608B880FB22E4F520D201D20043
:20020E00D203D205C2B4E4F50EF50DF50CF50BE4F512F511F510F50F74FFF513E588543F4F
:20022E00F588E589540FF5894420F5897450F598E5874480F58774FAF58BF58DD28ED2ACB7
:20024E0022C0E0C0D0C083C082309839E50DB4FA028030502E050DE50DB50E028004400259
:20026E00F50E90A000C0E0E50B2582F582E43583F583D0E0E599F0050BE50BB4FA0040036C
:20028E00750B00C298309948E511700DD200300235E4D5E0FDC2B4802DC20030011A3002C1
:2002AE0002D2B490A0FAC0E0E5102582F582E43583F583D0E0E0F59915110510E510B4FABB
:2002CE00004003751000C299200105200002D299D082D083D0D0D0E0322278FB120044E642
:2002EE00C0E0B40A0B300308D204740D1581C0E0E511B4FA0280F950F7C2AC90A0FAC0E021
:20030E00E50F2582F582E43583F583D0E0D0E0C0E0F00511050FE511B512004002F512E5A4
:20032E000FB4FA004003750F00300002D299D2ACD0E0300408C204740AC0E080B322E4F512
:20034E00F078FB120044F608A6F022E51364FF7038E50D6034300531C2AC90A000C0E0E50E
:20036E000C2582F582E43583F583D0E0E0D2ACB40A0302038774018010150D050CE50CB4F9
:20038E00FA004003750C0080C875F00022E4A20192E0F51F70030203BCE51160030203A77C
:2003AE00E4A20092E0F51FE51F70030203AE22C2AC7513FF750C00750B00E50D750D00D29B
:2003CE00AC75F0002274FFC513B4FF2EE50D0060FBC2AC90A000C0E0E50C2582F582E435FD
:2003EE0083F583D0E0E0C0E0150D050CE50CB4FA004003750C00D2ACD0E030050BB40A03FF
:20040E000203DAB40D02740A75F000221203D3C0E0C0E0C0E01202E8D0E0D0E0D0E075F0EE
:20042E000022E51375F0007BFF7C00120170700302044874FFF5F002045878FB120044E690
:20044E000886F0F51318E60886F02278FB1200448682088683E06016C083C082C0E0C0E06D
:20046E001202E8D0E0D0E0D082D083A380E722E4F5F078FB120044F608A6F02274F975F027
:20048E0052C0E0C0F0E52075F000C0E0C0F07402124ACC1581158115811581741475F053BC
:2004AE00C0E0C0F0E50F75F000C0E0C0F0E510C0E0C0F0E51175F000C0E0C0F0E512C0E0AE
:2004CE00C0F0740575F000124ACC7FF6120050744775F053C0E0C0F0E50B75F000C0E0C009
:2004EE00F0E50CC0E0C0F0E50D75F000C0E0C0F0E50EC0E0C0F0740575F000124ACC7FF658
:20050E00120050E4F50EF512227FFD7EFF1201EFE4F5F07F001201D3F0A3C5F0F0C5F078CD
:20052E00FB120044E60886F012013B18F608A6F012012D45F060221818188601088602891F
:20054E00828A8312007189828A83E012008BC0E0C0F0124BCB1581158145F070030206236F
:20056E007F001201D3E0A3F5F0E0C5F07B047C0012010D7F001201D3F0A3C5F0F0C5F07826
:20058E00F9120044860108860289828A8312007189828A83E012008BC0E0C0F0124BDA151B
:2005AE008115817F021201D3F07F021201D3E012008B7B3912007F12015A600B7F0212012A
:2005CE00D3E0C39430800B7F021201D3E0C39441240A75F0007F001201D312006A2BC5F015
:2005EE003CC5F07F001201D3F0A3C5F0F0C5F078F9120044860108860289828A83E0A3F53C
:20060E00F0E0C5F012012D89828A83F0A3C5F0F0C5F002052D7F001201D3E0A3F5F0E0C55C
:20062E00F07F030201ED7FF17EFF1201EF7F021201E1E98AF0C0E0C0F0E4C0E0C0E0740A91
:20064E0075F000C0E0C0F0124C0C7FFA1200507F021201E1E98AF07F0C1201D3F0A3C5F001
:20066E00F0C5F074097F0E1201D3F078FB120044860108860289828A8312007189828A8354
:20068E00E012008BC0E0C0F0124B921581158145F0602E78FB120044860108860289828A2C
:2006AE008312007189828A83E012008BC0E0C0F0124BC61581158145F060067F0E1201D3E4
:2006CE00E070030207437F0C1201D3E0A3F5F0E0C5F012012D7F0C1201D3F0A3C5F0F0C551
:2006EE00F012013BF9AAF0C001C00278F9120044860108860289828A8312007189828A8307
:20070E00E0D083D082F018860108860289828A83E0A3F5F0E0C5F012012D89828A83F0A327
:20072E00C5F0F0C5F07F0E1201D3E0147F0E1201D3F00206797F021201E1E98AF0C0E0C0CE
:20074E00F0124C2F158115817F001201D3F0A3C5F0F0C5F07F0F0201ED7FFE7EFF1201EF16
:20076E00E4F5F07F001201D3F0A3C5F0F0C5F07F001201D3E0A3F5F0E0C5F012014E45F058
:20078E00601B78FB120044E60886F012013B18F608A6F012012D7B007C0012016245F07058
:2007AE000302080D78F7120044E60886F012012D18F608A6F012013BF9AAF089828A83E023
:2007CE0012008BC0E0C0F008E60886F012012D18F608A6F012013BF9AAF089828A83E012DB
:2007EE00008BFBACF0D0F0D0E0C39BC5F09CC5F07F001201D3F0A3C5F0F0C5F002077D7F9E
:20080E00001201D3E0A3F5F0E0C5F07F020201ED7FFF7EFF1201EFE47F001201D3F07F00C1
:20082E001201D3E075F0007B107C00120187701202088D7F001201D3E0047F001201D3F027
:20084E0080DC78FB120044E60886F07F001201D31200662BC5F03400C5F0F9AAF07F001237
:20086E0001D3E0C001C00279567AA412008B12007889828A83E0F4D083D082F002084174DF
:20088E000190A47AF07F010201ED7FFF7EFF1201EFE4F521E4F5F090A2BEF0A3C5F0F0C58E
:2008AE00F0E490A2BDF074F475F0A1C0E0C0F0E4C0E0C0E074C975F000C0E0C0F0124C0C39
:2008CE007FFA120050E4F5F090A389F0A3C5F0F0C5F074C075F0A2C0E0C0F0E4C0E0C0E00E
:2008EE0074C975F000C0E0C0F0124C0C7FFA120050E490A455F0748C75F0A3C0E0C0F0E41A
:20090E00C0E0C0E074C975F000C0E0C0F0124C0C7FFA120050740190A47AF0E47F001201C9
:20092E00D3F07F001201D3E075F0007B107C00120181701202099E7F001201D3E0047F00AE
:20094E001201D3F080DC7F001201D3E079567AA412008B1200787F001201D3E0C001C00236
:20096E0079687AA412008B12007889828A83E0F412008BD083D08212006612007F12017881
:20098E00700302099BE490A47AF002099E02094590A47AE060030209E3745675F0A4C0E063
:2009AE00C0F0E4C0E0C0E0741275F000C0E0C0F0124C0C7FFA120050745675F0A4C0E0C0A2
:2009CE00F0749775F051C0E0C0F0124C781581158115811581121760121764746875F0A4DF
:2009EE00C0E0C0F012081E158115817F010201ED12039B78FB120044E60886F090A38BF03A
:200A0E00C209C2B490A38BE075F000900A3C020096E490A38BF0D208C202E490AEBBF00217
:200A2E000A50C208D202E490AEBBF0020A50300A0300300A0200300A0100240A00000000A5
:200A4E001F0A227FFB7EFF1201EF78F9120044E60886F07F031201D3F0A3C5F0F0C5F008BC
:200A6E00E60886F07F011201D3F0A3C5F0F0C5F07F011201E1E98AF0C0E0C0F0740275F0AF
:200A8E0000C0E0C0F012051715811581158115817F001201D3F078FB120044E60886F0C030
:200AAE00E0C0F0743075F000C0E0C0F07402C0E0C0F0124C0C7FFA1200507F031201D312BA
:200ACE00007189828A83E07003020B147F031201D31200717F001201D3E089828A831200B1
:200AEE00662B7F001201D3F07F031201D3E0A3F5F0E0C5F012012D7F031201D3F0A3C5F0AD
:200B0E00F0C5F0020AC87F001201D3E0F4047F001201D3F078FB12004486010886027F005D
:200B2E001201D3E075F0007B047C0012011BC001C00290519C12007112007889828A83E04E
:200B4E00D083D082F078FB120044E60886F02401C5F03400C5F0F9AAF07F001201D3E054D6
:200B6E000FC001C00290519C12007112008B12007889828A83E0D083D082F07F001201D3BC
:200B8E00E012008B54FFC5F05400C5F07F050201ED90A455E06003020C45748C75F0A3C05E
:200BAE00E0C0F0E4C0E0C0E074C975F000C0E0C0F0124C0C7FFA12005090A38BE075F00039
:200BCE007B007C0012018F7003020C31798C7AA3742489828A83F0E4A20992E0F51F748CE5
:200BEE0075F0A3C0E0C0F0E51F6007748B75F0538005748F75F053C0E0C0F0124C68158181
:200C0E00158115811581748C75F0A3C0E0C0F0745675F0A4C0E0C0F0124C68158115811582
:200C2E00811581748C75F0A3C0E0C0F0124CA61581158190A455F078FB120044E60886F061
:200C4E007B0A7C00120170700C18E60886F07BFF7C0012017045F07003020CD6E4A20992E4
:200C6E00E0F51F7003020C99748C75F0A3C0E0C0F0748C75F0A32401C5F03400C0F0C0E09A
:200C8E00120A511581158115811581748C75F0A3C0E0C0F01204591581158178FB120044C5
:200CAE00E60886F07B0A7C001201707003020CCE740A75F000C0E0C0F01202E81581158194
:200CCE00E490A455F0020D02748C75F0A390A4551200662BC5F03400C5F0F9AAF078FB12AE
:200CEE000044E60886F089828A83F090A455E00490A455F02278FB120044860108860289C5
:200D0E00828A83E07003020D4418860108860289828A83E012008BC0E0C0F0120B9F15812A
:200D2E00158178FB120044E60886F012012D18F608A6F0020D03227FFA7EFF1201EFE4F5F1
:200D4E00F07F021201D3F0A3C5F0F0C5F078FB120044E60886F07F001201D3F0A3C5F0F077
:200D6E00C5F0E47F041201D3F07F041201D3E075F0007B027C001201817003020FC57F046C
:200D8E001201D3E075F000900F9B020096C2097F001201D3E0A3F5F0E0C5F012012D7F005C
:200DAE001201D3F0A3C5F0F0C5F012013BF9AAF089828A83E012008B900F120200967F0014
:200DCE001201D312007189828A83E012008B7B2012007F1201707003020DF474017F0412D8
:200DEE0001D3F0020DFC74037F041201D3F0020F1E78FB120044E60886F0C0E0C0F018E69C
:200E0E000886F02401C5F03400C0F0C0E0120A5115811581158115817F051201D3F07F0545
:200E2E001201D3E07003020EB274037F041201D3F0742F75F075C0E0C0F090A2BEE0A3F5A4
:200E4E00F0E0C5F012012D90A2BEF0A3C5F0F0C0F0C0E0124CED158115811581158190A272
:200E6E00BEF0A3C5F0F0C5F090A38BE075F0007B027C001201707003020EAF749175F0534B
:200E8E00C0E0C0F07F051201D3E075F000C0E0C0F0740275F000124ACC158115811581151B
:200EAE0081020F047F001201D3E0A3F5F0E0C5F02402C5F03400C5F07F001201D3F0A3C5AB
:200ECE00F0F0C5F07F001201D312007189828A83E012008B7B2012007F1201707003020EC0
:200EEE00FC74017F041201D3F0D209020F0474037F041201D3F0020F1E74037F041201D34B
:200F0E00F0020F1EFF0D2300CC0D21000000070F020FA7745675F0A4C0E0C0F07F001201F8
:200F2E00D3E0A3F5F0E0C0F0C0E0745675F0A4C0E0C0F0124CA615811581C0E0C0F012077C
:200F4E00677FFA12005045F07003020F6674037F041201D3F0020F9874027F041201D3F0DA
:200F6E00745675F0A4C0E0C0F0124CA6158115817F001201D312006A2BC5F03CC5F07F02DD
:200F8E001201D3F0A3C5F0F0C5F0020FA7210F01009B0D00000000A70F7F001201D3E0A341
:200FAE00F5F0E0C5F012012D7F001201D3F0A3C5F0F0C5F0020D777F021201D3E0A3F5F0C2
:200FCE00E0C5F07F060201ED7FFD7EFF1201EFE4F5F07F011201D3F0A3C5F0F0C5F01203CD
:200FEE005945F070030212791203D37F001201D3F0E4A20892E0F51F700302101F7F0012CF
:20100E0001D3E012008BC0E0C0F01202E81581158190A2BDE0600302104774F475F0A1C040
:20102E00E0C0F0E4C0E0C0E074C975F000C0E0C0F0124C0C7FFA1200507F001201D3E01260
:20104E00008B9010BF02009690A2BDE0700302107890A2BDE01490A2BDF079F47AA11200D8
:20106E008B120078E489828A83F00210CB0210CB74F475F0A190A2BD1200662BC5F03400BE
:20108E00C5F0F9AAF07F001201D3E089828A83F090A2BDE00490A2BDF075F0007BC87C00D7
:2010AE0012019770030210BC74C790A2BDF00210CB7B100A005610080000007E107F00121E
:2010CE0001D3E012008B7B0A12007F120170700302127990A38BE075F0009012600200967B
:2010EE0079F47AA189828A83E012008B7B2A12007F120178700302111874F475F0A17F0178
:20110E001201D3F0A3C5F0F0C5F002127474F475F0A1C0E0C0F0120D45158115817F011286
:20112E0001D3F0A3C5F0F0C5F002127490A2BDE070030211B779F47AA189828A83E01200BA
:20114E008B9011A70200960211B774A875F053C0E0C0F01204591581158174F475F0A1C05F
:20116E00E0C0F01204591581158174AA75F053C0E0C0F01204591581158174F475F0A1C047
:20118E00E0C0F0120D45158115817F011201D3F0A3C5F0F0C5F00211B755112D0055112AE1
:2011AE0000551124000000581102127490A2BDE0700302124A79F47AA189828A83E0120074
:2011CE008B90123A02009602124A74F475F0A1C0E0C0F0120D45158115817F011201D3F000
:2011EE00A3C5F0F0C5F07F011201D3E0A3F5F0E0C5F045F0700302123774AC75F053C0E016
:20120E00C0F012045915811581745675F0A4C0E0C0F01204591581158174B075F053C0E03B
:20122E00C0F01204591581158102124AD5112D00D5112A00D51124000000D81102127474E5
:20124E000175F000C0E0C0F01209FE15811581021274BA1103003A1102001B110100EE10B7
:20126E00000000004D12E490A2BDF07F011201D3E0A3F5F0E0C5F07F030201ED90A38BE0CB
:20128E0075F0007B007C00120170700E90A38BE075F0007B027C0012017045F070030212A8
:2012AE00C378FB120044E60886F0C0E0C0F0120D03158115812290A38BE075F0007B007C76
:2012CE000012017070030212F7745675F0A4C0E0C0F01204591581158174B475F053C0E0C1
:2012EE00C0F012045915811581227FFD7EFF1201EF78FB120044E60886F02401C5F034003D
:20130E00C5F0F9AAF089828A83E012008B7B3D12007F120170700302145318E60886F0249A
:20132E0002C5F03400C5F07F001201D3F0A3C5F0F0C5F07F001201D3E0A3F5F0E0C0F0C090
:20134E00E0124CA6158115817B017C0012016A7003021440745675F0A4C0E0C0F0E4C0E08A
:20136E00C0E0741275F000C0E0C0F0124C0C7FFA120050E47F021201D3F07F021201D3E0BD
:20138E0075F0007B107C00120181600D7F001201D312007189828A83E070120213FD7F02DD
:2013AE001201D3E0047F021201D3F080CD7F021201D3E079567AA412008B1200787F0012C5
:2013CE0001D3E0A3F5F0E0C5F012012D7F001201D3F0A3C5F0F0C5F012013BC001C002F9D2
:2013EE00AAF089828A83E0D083D082F00213AC745675F0A4C0E0C0F0745675F0A4C0E0C0A1
:20140E00F0124CA615811581D004D0032BC5F03CC5F0F9AAF0742089828A83F012176074FA
:20142E006875F0A4C0E0C0F012081E1581158102145074B675F053C0E0C0F012128A15819D
:20144E00158102149E121760746875F0A4C0E0C0F012081E1581158174C075F0A2C0E0C077
:20146E00F074D075F053C0E0C0F0745675F0A4C0E0C0F0740375F000124AE37FFA12005009
:20148E0074C075F0A2C0E0C0F0120D03158115817F030201ED78FB120044E60886F018F6B8
:2014AE0008A6F074C075F0A2C0E0C0F074E375F053C0E0C0F0745675F0A4C0E0C0F07403FC
:2014CE0075F000124AE37FFA12005074C075F0A2C0E0C0F0120D0315811581788018E66050
:2014EE00FC881F74C075F0A2C0E0C0F074F475F053C0E0C0F0E51F75F000C0E0C0F0747F94
:20150E00C0E0C0F0740475F000124AE37FF812005074C075F0A2C0E0C0F0120D0315811520
:20152E00812278FB120044E60886F018F608A6F074C075F0A2C0E0C0F0740E75F054C0E0BB
:20154E00C0F0E50A75F000C0E0C0F090A2BEE0A3F5F0E0C0F0C0E0740475F000124AE37F06
:20156E00F812005074C075F0A2C0E0C0F0120D0315811581E4F50AE4F5F090A2BEF0A3C536
:20158E00F0F0C5F0227FFE7EFF1201EF78FB120044E60886F02401C5F03400C5F07F001209
:2015AE0001D3F0A3C5F0F0C5F07F001201D312007189828A83E012008BC0E0C0F0124BC66C
:2015CE001581158145F070030215F57F001201D3E0A3F5F0E0C0F0C0E0124C2F1581158167
:2015EE0090AEBBF002162F74C075F0A2C0E0C0F0743D75F054C0E0C0F090AEBBE075F0002A
:20160E00C0E0C0F0740375F000124AE37FFA12005074C075F0A2C0E0C0F0120D031581151E
:20162E00817F020201ED7FFE7EFF1201EF78FB120044E60886F02401C5F03400C5F07F003F
:20164E001201D3F0A3C5F0F0C5F07F001201D312007189828A83E012008B901703020096EA
:20166E0074C075F0A2C0E0C0F0745175F054C0E0C0F090A38BE075F000C0E0C0F0740375C4
:20168E00F000124AE37FFA12005074C075F0A2C0E0C0F0120D031581158102170B7F0012A4
:2016AE0001D312007189828A83E012008BC0E0C0F0124BC61581158145F070030216F07F62
:2016CE00001201D3E0A3F5F0E0C0F0C0E0124C2F15811581C0E0C0F01209FE15811581022E
:2016EE001700746175F054C0E0C0F012128A1581158102170B6E1600000000AB167F020221
:20170E0001ED90A38BE075F0007B007C00120170700302175F74C075F0A2C0E0C0F07479ED
:20172E0075F054C0E0C0F078F7120044E60886F0C0E0C0F0740375F000124AE37FFA120073
:20174E005074C075F0A2C0E0C0F012128A1581158122E4F5F022D290A290B3E492E0F51F08
:20176E00E51F7003021784E4C0E0C0E01209FE15811581021794740175F000C0E0C0F012F5
:20178E0009FE15811581227FFA7EFF1201EF78FB120044E60886F07F021201D3F0A3C5F012
:2017AE00F0C5F07F001201D3F0A3C5F0F0C5F07F001201D312007189828A83E070030218B7
:2017CE006F7F001201D312007189828A83E012008B7B2012007F120170700302180A7F004A
:2017EE001201D3E0A3F5F0E0C5F012012D7F001201D3F0A3C5F0F0C5F002186C7F0212014C
:20180E00D3120071C001C0027F001201D312007189828A83E012008BC0E0C0F0124BDA15C8
:20182E00811581D083D082F07F001201D3E0A3F5F0E0C5F012012D7F001201D3F0A3C5F09F
:20184E00F0C5F07F021201D3E0A3F5F0E0C5F012012D7F021201D3F0A3C5F0F0C5F00217C4
:20186E00BD7F021201D3120071E489828A83F078FB120044E60886F02401C5F03400C5F0D7
:20188E007F001201D3F0A3C5F0F0C5F018860108860289828A83E012008B901EFF020096DF
:2018AE0078FB120044E60886F0C0E0C0F01212F815811581021F371214A3123986021F370B
:2018CE0078FB120044E60886F0C0E0C0F012153015811581021F37122A86122A76021F37D6
:2018EE0078FB120044E60886F0C0E0C0F012159315811581021F377F001201D312007189AE
:20190E00828A83E012008BC0E0C0F0124BC61581158145F070030219437F001201D3E0A320
:20192E00F5F0E0C0F0C0E0124C2F1581158190ACB4F002197D74C075F0A2C0E0C0F07494C0
:20194E0075F054C0E0C0F090ACB4E075F000C0E0C0F0740375F000124AE37FFA1200507481
:20196E00C075F0A2C0E0C0F0120D0315811581021F3778FB120044E60886F0C0E0C0F0120D
:20198E00163415811581021F37E4A21692E0F51F74C075F0A2C0E0C0F074B475F054C0E03D
:2019AE00C0F0E51F75F000C0E0C0F07403124AE37FFA12005074C075F0A2C0E0C0F0120D75
:2019CE000315811581E4A21592E0F51F74C075F0A2C0E0C0F074BD75F054C0E0C0F0E51FE0
:2019EE0075F000C0E0C0F07403124AE37FFA12005074C075F0A2C0E0C0F0120D031581153B
:201A0E0081C215021F377F001201D312007189828A83E012008B901B2102009674FF75F04F
:201A2E0000C0E0C0F0E4C0E0C0F012308A1581158115811581021B2D74FE75F000C0E0C06F
:201A4E00F0E4C0E0C0F012308A1581158115811581021B2D7F001201D312007189828A83E6
:201A6E00E07003021B1E7F001201E1E98AF0C0E0C0F0121F3C158115817F041201D3F0A30F
:201A8E00C5F0F0C5F07F041201D3E0A3F5F0E0C5F012014E45F0703A7F041201D3E0A3F557
:201AAE00F0E0C5F07B027C00120170600E90A47CE075F0007BFF7C0012017045F070137F04
:201ACE00041201D3E0A3F5F0E0C5F07B037C0012017045F07003021B0B90A47BE075F000D0
:201AEE00C0E0C0F090A47CE075F000C0E0C0F012308A1581158115811581021B1B74C1753D
:201B0E00F054C0E0C0F012128A15811581021A62021B2D461A53002A1A00000000621A020C
:201B2E001F377F001201D312007189828A83E012008B901C9202009674C075F0A2C0E0C053
:201B4E00F074D975F054C0E0C0F090ACB5E0A3F5F0E0C0F0C0E0123E81C0E0C0F07404759A
:201B6E00F000124AE37FF812005074C075F0A2C0E0C0F0120D0315811581021CAA7F00121D
:201B8E0001D3E0A3F5F0E0C5F02401C5F03400C0F0C0E0124C2F158115817B3C7C0012000A
:201BAE00C0C0E0C0F01246DB15811581021CAA7F001201D3E0A3F5F0E0C0F0C0E074FF75FB
:201BCE00F054C0E0C0F0124D34158115811581158145F07003021BF9740475F055C0E0C028
:201BEE00F012128A15811581021BFF12039B020000021CAA123F66021CAA7F001201D3E0B3
:201C0E00A3F5F0E0C5F02401C5F03400C0F0C0E0124C2F15811581C0E0C0F01246B1158193
:201C2E001581021CAA7F001201D312007189828A83E012008BC0E0C0F0124BC6158115811C
:201C4E0045F07003021C7F7F001201D3E0A3F5F0E0C0F0C0E0124C2F158115817B3C7C0048
:201C6E001200C0C0E0C0F01246B115811581021C8F741975F055C0E0C0F012128A15811562
:201C8E0081021CAA081C5300021C5100BD1B45008B1B4300461B00000000331C021F377F7A
:201CAE00001201D312007189828A83E07003021D6F7F001201E1E98AF0C0E0C0F0121F3C21
:201CCE00158115817F041201D3F0A3C5F0F0C5F07F041201D3E0A3F5F0E0C5F045F0700366
:201CEE00021D04743175F055C0E0C0F012128A15811581021D6C90A47BE075F000C0E0C04B
:201D0E00F090A47CE075F000C0E0C0F090A47DE075F000C0E0C0F090A47EE075F000C0E0A3
:201D2E00C0F01236287FF812005090A47BE075F000C0E0C0F090A47CE075F000C0E0C0F013
:201D4E0090A47DE075F000C0E0C0F090A47EE075F000C0E0C0F01241287FF8120050021C76
:201D6E00AD021F37021F37744975F055C0E0C0F0120D0315811581747F75F055C0E0C0F0E6
:201D8E00120D031581158174A275F055C0E0C0F0120D031581158174DE75F055C0E0C0F01D
:201DAE00120D0315811581740875F056C0E0C0F0120D0315811581742F75F056C0E0C0F044
:201DCE00120D0315811581745E75F056C0E0C0F0120D0315811581748C75F056C0E0C0F071
:201DEE00120D031581158174AC75F056C0E0C0F0120D031581158174DF75F056C0E0C0F0B0
:201E0E00120D031581158174FF75F056C0E0C0F0120D0315811581742D75F057C0E0C0F0ED
:201E2E00120D0315811581745D75F057C0E0C0F0120D0315811581748475F057C0E0C0F017
:201E4E00120D031581158174A975F057C0E0C0F0120D031581158174CF75F057C0E0C0F060
:201E6E00120D0315811581740375F058C0E0C0F0120D0315811581742975F058C0E0C0F08A
:201E8E00120D0315811581745375F058C0E0C0F0120D0315811581748875F058C0E0C0F0BB
:201EAE00120D031581158174BB75F058C0E0C0F0120D031581158174F275F058C0E0C0F0C9
:201ECE00120D0315811581741175F059C0E0C0F0120D0315811581021F3778FB120044E6BE
:201EEE000886F0C0E0C0F012171015811581021F37751D3F00721D0000AD1C5300301B5230
:201F0E0000141A51009719500080194E0005194D00EE184C00E5184600CE184500C5184401
:201F2E0000AE1841000000E81E7F060201ED7FFA7EFF1201EFE4F5F07F041201D3F0A3C58F
:201F4E00F0F0C5F0E4F5F07F001201D3F0A3C5F0F0C5F078FB120044860108860289828A4E
:201F6E0083E0A3F5F0E0C5F07F021201D3F0A3C5F0F0C5F0740290A47EF074FF90A47CF054
:201F8E007F021201D312007189828A83E012008B45F060267F041201D3E0A3F5F0E0C5F093
:201FAE0012014E45F060137F001201D3E0A3F5F0E0C5F07B047C0012015445F0700302227A
:201FCE00497F001201D3E0A3F5F0E0C5F09022320200967F021201D312007189828A83E0EA
:201FEE0012008B7B4112007F12016A60187F021201D312007189828A83E012008B7B501298
:20200E00007F12015A45F070030220677F021201D312007189828A83E0C3944190A47BF07C
:20202E007F021201D3E0A3F5F0E0C5F012012D7F021201D3F0A3C5F0F0C5F07F001201D335
:20204E00E0A3F5F0E0C5F012012D7F001201D3F0A3C5F0F0C5F0022078740175F0007F04EC
:20206E001201D3F0A3C5F0F0C5F00222467F021201D3E0A3F5F0E0C0F0C0E01238831581B3
:20208E00158190A47CF07B007C00120197600E90A47CE075F0007B107C0012018145F070B8
:2020AE00030220F07F021201D3E0A3F5F0E0C5F02402C5F03400C5F07F021201D3F0A3C516
:2020CE00F0F0C5F07F001201D3E0A3F5F0E0C5F012012D7F001201D3F0A3C5F0F0C5F00267
:2020EE002101740275F0007F041201D3F0A3C5F0F0C5F00222467F021201D3E0A3F5F0E066
:20210E00C0F0C0E01238831581158190A47DF075F0007BFF7C00120178600E90A47DE0756D
:20212E00F0007B107C0012019745F0700302217C7F021201D3E0A3F5F0E0C5F02402C5F06A
:20214E003400C5F07F021201D3F0A3C5F0F0C5F07F001201D3E0A3F5F0E0C5F012012D7F13
:20216E00001201D3F0A3C5F0F0C5F002218D740375F0007F041201D3F0A3C5F0F0C5F0029A
:20218E0022467F021201D312007189828A83E012008BC0E0C0F0124BC61581158145F07006
:2021AE000302220E7F021201D3E0A3F5F0E0C0F0C0E0124C2F1581158190A47EF07F0212EF
:2021CE0001D312007189828A83E012008BC0E0C0F0124BC61581158145F0700302220B7F10
:2021EE00021201D3E0A3F5F0E0C5F012012D7F021201D3F0A3C5F0F0C5F00221CB02221432
:20220E00740290A47EF07F001201D3E0A3F5F0E0C5F012012D7F001201D3F0A3C5F0F0C594
:20222E00F002224690210300042102007B200100E11F000000004622021F8E7F021201D341
:20224E0012007189828A83E012008B45F060187F021201D312007189828A83E012008B7BB1
:20226E002C12007F12017845F0700302229A7F021201D3E0A3F5F0E0C5F012012D7F02126B
:20228E0001D3F0A3C5F0F0C5F00222497F021201D312007189828A83E012008B7B2C1200CA
:2022AE007F12017070030222D27F021201D3E0A3F5F0E0C5F012012D7F021201D3F0A3C542
:2022CE00F0F0C5F078FB12004486010886027F021201D3E0A3F5F0E0C5F089828A83F0A36C
:2022EE00C5F0F0C5F07F041201D3E0A3F5F0E0C5F07F060201EDE4F523F522E4F514E49027
:20230E00ACB3F074B375F0AAC0E0C0F0E4C0E0C0E0E475F001C0E0C0F0124C0C7FFA120027
:20232E005074B375F0ABC0E0C0F0E4C0E0C0E0E475F001C0E0C0F0124C0C7FFA120050E4D1
:20234E00F518747C75F04FF51985F01AE51875F000C333C5F033C5F0797C7A4F120078895B
:20236E00828A83E0A3F5F0E0C5F0F51B85F01CE4F515E4F517F516D295742775F000C0E032
:20238E00C0F0E4C0E0C0E0740475F000C0E0C0F0124D6A7FFA120050747F75F0A4C0E0C02E
:2023AE00F0E4C0E0C0E074F475F005C0E0C0F0124C0C7FFA120050E4F52EF52DF52CF52B2A
:2023CE00747F75F0A4F52485F025747375F0AAC0E0C0F0E4C0E0C0E0744075F000C0E0C05D
:2023EE00F0124C0C7FFA120050E4F531E4F535F534F533F532740190ACB4F0E58854CFF530
:20240E0088E58954F0F5894401F589E4F58AF58CD2B9D2A9D28CD288D2A822D294C0E0C02F
:20242E00D0A212B392B3C28C851B8A851C8CD28CC0F0C083C082C000E518B41500401643BB
:20244E000A02904F7C85821985831AE0F51BA3E0F51CE4F51825E02481F58274243400F56E
:20246E0083E0F5F0A3E0C0E0C0F0E527A2E7821392122224AF24BA24C424C724CA24CF24BA
:20248E00D224D524DA25022505250C25162519251C252125242527252C255025CE00000095
:2024AE0000B294B294A21E921F0226D9A2B5B3921EC2120226D90226D90226D9C212022683
:2024CE00D90226D90226D9C2120226D9301322E52A33F52AE52933F529E52833F528E527B0
:2024EE0033F527E52A92E0F52AC212E526600215260226D90225E9A21E921F0226D9A2B589
:20250E00B3921EC2120226D90226D90226D9C2120226D90226D90226D9C2120226D9301384
:20252E001EE52A33F52AE52933F529E52833F528E52733F527E52A92E0F52AC21215260246
:20254E0026D9201310E52D70030225CB8524828525830225ABE52660030225CB852482857A
:20256E002583E0430A106007530AEF14F0702EE52C04B4FE004001E4F52C75F006A4247F54
:20258E00F582E5F034A4F583858224858325152DE52D7009C213C212D2960225CBA3E0F5F1
:2025AE0026A375F0047827E0F6A308D5F0F9E527A2E79212D213C296B29600B2960225E9E7
:2025CE00B294751800904F7C85821985831AB294B294D214D289B2940226E9301D05C21D28
:2025EE00022674E531B40A0280044002740B25E09026160531D21DA21EB01F92D5A21FB0B9
:20260E001E72D592D5A21F738016801C80288030803880408053805B8063806B8073803E7D
:20262E00301F3E301E3B803E301F36201E33752F00753000803030D528E53033F530802689
:20264E0030D51EE53033F530801C30D514E53033F530801230D50AE53033F5308008430AD7
:20266E0004753100C21D0226D930D5F5E52F33F52F80F330D5EBE52F33F52F80E930D5E140
:20268E00E52F33F52F80DF30D5D7E52F33F52F80D530D5CDE52F33F52F90AA73E53225E0C0
:2026AE002582F582E43583F583E52FF0A3E530F00534E534B5350280044002F5350532E5E4
:2026CE0032B42000400375320080960518851A83851982A3A385831A858219E0F51BA3E08C
:2026EE00F51CD000D082D083D0F0D0D0D0E0C2943222D293C0E0C0F0C0D0C083C082A2120E
:20270E00B392B37400B518028012F518904F7C85831A858219E0F51BA3E0F51CD28DE51557
:20272E00B4020280044002740325E090273D73800680168040805B2014030227A8751501E0
:20274E007516007517010227A82014120516751700E516B41E0040427515000227A8751660
:20276E00000517E517B41E004030D216D215C29575150280252014157517000516E516B4FB
:20278E001E004016751500C216D295800D7516008008751500430A018000C214C2890514BC
:2027AE00E514B43C004005751400D217D082D083D0D0D0F0D0E0C293322274C075F0A2C012
:2027CE00E0C0F0742D75F059C0E0C0F078F7120044E60886F02441C5F03400C0F0C0E018CD
:2027EE00E60886F07B057C001200C02404C5F03400C5F079AC7A4F12007889828A83E075EE
:20280E00F000C0E0C0F0740475F000124AE37FF812005074C075F0A2C0E0C0F0120D0315B3
:20282E008115812274C075F0A2C0E0C0F0743575F059C0E0C0F078F7120044E60886F07B6B
:20284E00057C001200C02404C5F03400C5F0790D7A5012007889828A83E075F000C0E0C0BA
:20286E00F0740375F000124AE37FFA12005074C075F0A2C0E0C0F0120D03158115812274F5
:20288E00C075F0A2C0E0C0F0743A75F059C0E0C0F078F7120044E60886F0C333C5F033C58B
:2028AE00F079CD7A5012007889828A83E0A3F5F0E0C0F0C0E0740375F000124AE37FFA122A
:2028CE00005074C075F0A2C0E0C0F0120D03158115812278FB120044E60886F079FC7A4F34
:2028EE0012007889828A83E0C3944112008B2278FB120044E60886F079AD7A5012007889C1
:20290E00828A83E075F000227FFE7EFF1201EFE5347003022A55E53375F000C333C5F0334F
:20292E00C5F079737AAA12007889828A83E0A3F5F0E0C5F07F001201D3F0A3C5F0F0C5F0D3
:20294E000533E533E53375F0007B207C001201977003022966E4F5331534E53490AEBBE090
:20296E00540175F0007B007C001201787003022A52743D75F059C0E0C0F0120D0315811590
:20298E00817F001201D3E0A3F5F0E0C5F05400C5F0540FC5F07B087C0012011BC0E0C0F0A8
:2029AE001228E115811581C0E0C0F01227C815811581744675F059C0E0C0F0120D031581C5
:2029CE0015817F001201D3E0A3F5F0E0C5F0541FC5F05400C5F07B007C0012011BC0E0C03B
:2029EE00F01228FD15811581C0E0C0F012283215811581744C75F059C0E0C0F0120D031589
:202A0E008115817F001201D3E0A3F5F0E0C5F0541FC5F05400C5F07B007C0012011BC0E039
:202A2E00C0F01228FD15811581C0E0C0F012288D15811581744F75F059C0E0C0F0120D033F
:202A4E0015811581022A6574FFF5F07F001201D3F0A3C5F0F0C5F07F001201D3E0A3F5F034
:202A6E00E0C5F07F020201ED1229167BFF7CFF1201786003022A7622C2A9C2A8C212C213CC
:202A8E00742775F000C0E0C0F0E4C0E0C0E0740475F000C0E0C0F0124D6A7FFA120050746F
:202AAE007F75F0A4C0E0C0F0E4C0E0C0E074F475F005C0E0C0F0124C0C7FFA120050E4F5CC
:202ACE002EF52DF52CF52B747F75F0A4F52485F025D296D2A8D2A9227FFD7EFF1201EF78B6
:202AEE00FB120044E60886F05400C5F0540FC5F07B087C0012011B79FC7A4F1200788982F2
:202B0E008A83E0C394417F011201D3F078FB120044E60886F0541FC5F05400C5F07B007C77
:202B2E000012011B79AD7A5012007889828A83E07F001201D3F090ACB3E075F000902D1B86
:202B4E000200967F001201D3E075F0007B107C001201817003022C13E47F021201D3F07F1C
:202B6E00021201D3E075F0007B107C001201817012022BE37F021201D3E0047F021201D33B
:202B8E00F080DC7F021201D3E075F0007F011201D31200667C001201787003022BE07F0249
:202BAE001201D3E075F0007B107C001200C079B37AAA120078E98AF0C0E0C0F0E4C0E0C032
:202BCE00E0741075F000C0E0C0F0124C0C7FFA120050022B827F011201D3E075F0007B10A4
:202BEE007C001200C07F001201D31200662BC5F03400C5F079B37AAA120078740189828AEF
:202C0E0083F0022C3E7F011201D3E075F000C0E0C0F07F001201D3E075F000C0E0C0F012C0
:202C2E002D2C1581158115811581740190ACB3F0022D277F001201D3E075F0007B107C007A
:202C4E001201817003022CA974B375F0AAC0E0C0F0E4C0E0C0E0E475F001C0E0C0F0124CE6
:202C6E000C7FFA1200507F011201D3E075F0007B107C001200C07F001201D31200662BC50E
:202C8E00F03400C5F079B37AAA120078740189828A83F0E490ACB3F0022CCE7F011201D3D1
:202CAE00E075F000C0E0C0F07F001201D3E075F000C0E0C0F0122D2C1581158115811581B4
:202CCE00022D27E50A4408F50AE490ACB3F074B375F0AAC0E0C0F0E4C0E0C0E0E475F0019F
:202CEE00C0E0C0F0124C0C7FFA12005074B375F0ABC0E0C0F0E4C0E0C0E0E475F001C0E09C
:202D0E00C0F0124C0C7FFA120050022D27412C0100512B00000000D12C7F030201ED7FFF83
:202D2E007EFF1201EF78FB120044E60886F090306D020096E47F001201D3F07F001201D376
:202D4E00E075F0007B107C001201817012022E017F001201D3E0047F001201D3F080DC7860
:202D6E00F9120044E60886F07B107C001200C07F001201D31200662BC5F03400C5F079B3E7
:202D8E007AAA12007889828A83E07003022DFE78F9120044E60886F07B107C001200C07F5C
:202DAE00001201D31200662BC5F03400C5F079B37AAB120078740289828A83F078F9120002
:202DCE0044E60886F0C0E0C0F07F001201D3E075F000C0E0C0F008E60886F0C0E0C0F074C3
:202DEE000275F000C0E0C0F01241287FF8120050022D5E023085E47F001201D3F07F0012AC
:202E0E0001D3E075F0007B107C001201817012022EBF7F001201D3E0047F001201D3F08061
:202E2E00DC78F9120044E60886F07B107C001200C07F001201D31200662BC5F03400C5F0FE
:202E4E0079B37AAA12007889828A83E07003022EBC78F9120044E60886F07B107C001200EF
:202E6E00C07F001201D31200662BC5F03400C5F079B37AAB120078740289828A83F078F914
:202E8E00120044E60886F0C0E0C0F07F001201D3E075F000C0E0C0F008E60886F0C0E0C054
:202EAE00F0E4C0E0C0E01241287FF8120050022E20023085E47F001201D3F07F001201D3F7
:202ECE00E075F0007B107C001201817012022F817F001201D3E0047F001201D3F080DC785E
:202EEE00F9120044E60886F07B107C001200C07F001201D31200662BC5F03400C5F079B366
:202F0E007AAA12007889828A83E07003022F7E78F9120044E60886F07B107C001200C07F58
:202F2E00001201D31200662BC5F03400C5F079B37AAB120078740189828A83F078F9120081
:202F4E0044E60886F0C0E0C0F07F001201D3E075F000C0E0C0F008E60886F0C0E0C0F07441
:202F6E000275F000C0E0C0F01241287FF8120050022EDE02308578F9120044E60886F0C088
:202F8E00E0C0F07F001201D3E075F000C0E0C0F008E60886F0C0E0C0F0E4C0E0C0E0124166
:202FAE00287FF8120050E47F001201D3F07F001201D3E075F0007B107C0012018170120200
:202FCE0030497F001201D3E0047F001201D3F080DC78F9120044E60886F07B107C0012002C
:202FEE00C07F001201D31200662BC5F03400C5F079B37AAB12007889828A83E075F0007BAA
:20300E00007C00120178700302304678F9120044E60886F07B107C001200C07F001201D347
:20302E001200662BC5F03400C5F079B37AAB120078740189828A83F0022FD074B375F0AAB2
:20304E00C0E0C0F0E4C0E0C0E0E475F001C0E0C0F0124C0C7FFA120050023085023085841D
:20306E002F1000C22E1300042E1500042E1400422D120000006A307F010201ED7FFC7EFFF0
:20308E001201EF78F9120044E60886F09033B5020096E4F5F078F9120044F608A6F078F950
:2030AE00120044E60886F07B107C0012018170160230F878F9120044E60886F012012D187A
:2030CE00F608A6F080D878F9120044E60886F0C0E0C0F074FF75F000C0E0C0F012308A1572
:2030EE00811581158115810230C10233C1E4F5F078F9120044F608A6F078F9120044E608BD
:20310E0086F07B107C00120181701602322E78F9120044E60886F012012D18F608A6F08011
:20312E00D8E4F5F07F001201D3F0A3C5F0F0C5F0E4F5F078FB120044F608A6F078FB1200E3
:20314E0044E60886F07B107C0012018170160231EE78FB120044E60886F012012D18F608F4
:20316E00A6F080D878F9120044E60886F07B107C001200C00826C5F00836C5F079B37AAB28
:20318E0012007889828A83E075F0007B027C001201706007740175F0008003E4F5F07F02B0
:2031AE001201D3F0A3C5F0F0C5F07F021201D3E0A3F5F0E0C5F078FB1200448603088604E6
:2031CE0012010D7F001201D312006A4BC5F04CC5F07F001201D3F0A3C5F0F0C5F002315FFB
:2031EE0074C075F0A2C0E0C0F0745275F059C0E0C0F07F001201D3E0A3F5F0E0C0F0C0E065
:20320E00740375F000124AE37FFA12005074C075F0A2C0E0C0F0120D031581158102311C82
:20322E00740A75F000C0E0C0F0120B9F158115810233C178FB120044E60886F07BFF7C004C
:20324E00120170700302332174C075F0A2C0E0C0F0745775F059C0E0C0F0181818E60886F4
:20326E00F02441C5F03400C0F0C0E0740375F000124AE37FFA12005074C075F0A2C0E0C021
:20328E00F0120D0315811581E4F5F078FB120044F608A6F078FB120044E60886F07B107C88
:2032AE0000120181701602330E78FB120044E60886F012012D18F608A6F080D878F91200AF
:2032CE0044E60886F07B107C001200C00826C5F00836C5F079B37AAB12007889828A83E0B6
:2032EE0079937A5112008B12007889828A83E012008BC0E0C0F0120B9F158115810232B70A
:20330E00740A75F000C0E0C0F0120B9F158115810233B274C075F0A2C0E0C0F0745B75F0DE
:20332E0059C0E0C0F078F5120044E60886F02441C5F03400C0F0C0E008E60886F02401C5BB
:20334E00F03400C0F0C0E0181818E60886F07B107C001200C00826C5F00836C5F079B37AEA
:20336E00AB12007889828A83E075F000C333C5F033C5F0798D7A5112007889828A83E0A324
:20338E00F5F0E0C0F0C0E0740575F000124AE37FF612005074C075F0A2C0E0C0F0120D0369
:2033AE00158115810233C1FB30FE00A030FF00000041327F040201ED7FFF7EFF1201EF788A
:2033CE00FB120044E60886F02402C5F03400C0F0C0E074A875F04FC0E0C0F0740475F000CE
:2033EE00C0E0C0F0124DC37FFA120050E47F001201D3F07F001201D3E075F0007B047C0094
:20340E00120181701302348C7F001201D3E0047F001201D3F01480DB78FB120044E608867B
:20342E00F02402C5F03400C5F07F001201D31200662BC5F03400C5F0F9AAF078F7120044CC
:20344E00E60886F07B057C001200C07F001201D31200662BC5F03400C5F0C001C00279ACDE
:20346E007A4F120078D083D082C082C083E089828A831200664BD083D082F0023416E47FC2
:20348E00001201D3F07F001201D3E075F0007B047C00120181701302351C7F001201D3E0F4
:2034AE00047F001201D3F01480DB78FB120044E60886F02402C5F03400C5F07F001201D3E0
:2034CE001200662BC5F03400C5F0F9AAF0181818E60886F07B057C001200C07F001201D32B
:2034EE001200662BC5F03400C5F0C001C002790D7A50120078D083D082C082C083E089820B
:20350E008A831200664BD083D082F00234A87F010201ED7FFF7EFF1201EFE52D75F0007BFB
:20352E00FE7C001201977003023550E50A4420F50AE52D75F0007BFE7C0012019760030292
:20354E00353F78F5120044E60886F0C0E0C0F008E60886F0C0E0C0F0E52B75F0007B067C44
:20356E00001200C02400C5F03400C5F0797F7AA4120078E98AF0C0E0C0F01233C67FFA12C0
:20358E000050E52B75F0007B067C001200C02400C5F03400C5F0797F7AA412007878FB12A2
:2035AE000044E60886F089828A83F0E52B75F0007B067C001200C02401C5F03400C5F079CD
:2035CE007F7AA412007878F9120044E60886F089828A83F0052BE52BE52B75F0007BFE7CD9
:2035EE000012019770030235FAE4F52B052DE52D7F001201D3F0E52E75F0007F001201D3F5
:20360E001200667C0012018170030236237F001201D3E0F52E7F010201ED90AEBBE054023F
:20362E0075F0007B007C00120178700302372D746675F059C0E0C0F0120D0315811581780E
:20364E00F5120044E60886F0C0E0C0F01227C815811581746F75F059C0E0C0F0120D031508
:20366E0081158178F7120044E60886F0C0E0C0F012283215811581747375F059C0E0C0F01F
:20368E00120D031581158178F9120044E60886F0C0E0C0F01228321581158174C075F0A280
:2036AE00C0E0C0F0747775F059C0E0C0F078F7120044E60886F0C0E0C0F0740375F000124C
:2036CE004AE37FFA12005074C075F0A2C0E0C0F0120D031581158178F7120044E60886F0D2
:2036EE00C0E0C0F012288D15811581742075F000C0E0C0F0120B9F1581158178F912004481
:20370E00E60886F0C0E0C0F012288D15811581748375F059C0E0C0F0120D03158115817829
:20372E00F5120044E60886F0C0E0C0F008E60886F0C0E0C0F0741675F000C0E0C0F074010C
:20374E00C0E0C0F01235217FF812005078F5120044E60886F0C0E0C0F008E60886F0C0E047
:20376E00C0F0742075F000C0E0C0F07401C0E0C0F01235217FF8120050740175F000C0E0C2
:20378E00C0F078F9120044E60886F0C0E0C0F0124CD1158115811581158178FB120044F6AA
:2037AE0008A6F074FF75F000C0E0C0F018E60886F0C0E0C0F0124CED1581158115811581C6
:2037CE0078FB120044F608A6F018E60886F07B017C00120170700302381A78F5120044E617
:2037EE000886F0C0E0C0F0080808E60886F0C0E0C0F0742075F000C0E0C0F07401C0E0C003
:20380E00F01235217FF812005002388278F5120044E60886F0C0E0C0F0080808E60886F0BA
:20382E00C0E0C0F0741675F000C0E0C0F008E60886F0C39401C5F09400C0F0C0E012352126
:20384E007FF812005078F5120044E60886F0C0E0C0F0080808E60886F0C0E0C0F074207535
:20386E00F000C0E0C0F07401C0E0C0F01235217FF8120050227FFD7EFF1201EF74FFF5F07F
:20388E007F011201D3F0A3C5F0F0C5F0E47F001201D3F07F001201D3E075F0007B207C00CD
:2038AE0012018170130239757F001201D3E0047F001201D3F01480DB7F001201D3E075F07C
:2038CE00007B037C001200C02400C5F03400C5F0790D7A51120078C001C00278F912004427
:2038EE008601088602D083D082E012008B89828A8312006612007F120170604C7F0012019F
:20390E00D3E075F0007B037C001200C02401C5F03400C5F0790D7A5112007878FB1200444E
:20392E00E60886F02401C5F03400C5F0C001C002F9AAF0D083D082E012008B89828A8312F0
:20394E00006612007F12017045F070030239727F001201D3E07F011201D3F0A3C5F0F0C5E2
:20396E00F00239750238B67F011201D3E0A3F5F0E0C5F07F030201ED7FFF7EFF1201EF7463
:20398E008675F059C0E0C0F0120D031581158174C075F0A2C0E0C0F0749A75F059C0E0C080
:2039AE00F0E52B75F000C0E0C0F0E52CC0E0C0F0E52D75F000C0E0C0F07405124AE37FF6EF
:2039CE0012005074C075F0A2C0E0C0F0120D031581158174C075F0A2C0E0C0F074C475F076
:2039EE0059C0E0C0F0E52E75F000C0E0C0F0E5248525F0C0E0C0F0E50A75F000C0E0C0F0B1
:203A0E007405124AE37FF6120050E4F50A74C075F0A2C0E0C0F0120D031581158174C075A4
:203A2E00F0A2C0E0C0F074EA75F059C0E0C0F0740275F000124AE315811581158115817444
:203A4E00C075F0A2C0E0C0F0120D0315811581E47F001201D3F07F001201D3E075F0007B95
:203A6E00067C001201817013023AE97F001201D3E0047F001201D3F01480DB74C075F0A232
:203A8E00C0E0C0F074FB75F059C0E0C0F0E52B75F0007B067C001200C07F001201D3120090
:203AAE00662BC5F03400C5F0797F7AA412007889828A83E075F000C0E0C0F0740375F000A0
:203ACE00124AE37FFA12005074C075F0A2C0E0C0F0120D0315811581023A7974C075F0A2F5
:203AEE00C0E0C0F0740175F05AC0E0C0F0740275F000124AE3158115811581158174C075C9
:203B0E00F0A2C0E0C0F0120D0315811581E47F001201D3F07F001201D3E075F0007B067C87
:203B2E00001201817013023BA77F001201D3E0047F001201D3F01480DB74C075F0A2C0E094
:203B4E00C0F0741375F05AC0E0C0F0E52C75F0007B067C001200C07F001201D31200662BC4
:203B6E00C5F03400C5F0797F7AA412007889828A83E075F000C0E0C0F0740375F000124A14
:203B8E00E37FFA12005074C075F0A2C0E0C0F0120D0315811581023B3774C075F0A2C0E031
:203BAE00C0F0741975F05AC0E0C0F0740275F000124AE3158115811581158174C075F0A2FE
:203BCE00C0E0C0F0120D0315811581E47F001201D3F07F001201D3E075F0007B067C001247
:203BEE0001817013023C5A7F001201D3E0047F001201D3F01480DB74C075F0A2C0E0C0F082
:203C0E00742B75F05AC0E0C0F0E5248525F07F001201D31200662BC5F03400C5F0F9AAF00C
:203C2E0089828A83E075F000C0E0C0F0740375F000124AE37FFA12005074C075F0A2C0E0F8
:203C4E00C0F0120D0315811581023BF574C075F0A2C0E0C0F0743175F05AC0E0C0F0740271
:203C6E0075F000124AE3158115811581158174C075F0A2C0E0C0F0120D0315811581E47FFE
:203C8E00001201D3F07F001201D3E075F0007B047C001201817013023CFF7F001201D3E002
:203CAE00047F001201D3F01480DB74C075F0A2C0E0C0F0744375F05AC0E0C0F07F0012014B
:203CCE00D3E079277A0075F000120078E775F000C0E0C0F07403124AE37FFA12005074C0B9
:203CEE0075F0A2C0E0C0F0120D0315811581023CA8740A75F000C0E0C0F0120B9F15811591
:203D0E008174C075F0A2C0E0C0F0744975F05AC0E0C0F0E53275F000C0E0C0F0E533C0E039
:203D2E00C0F0E53475F000C0E0C0F0E535C0E0C0F0740675F000124AE37FF412005074C066
:203D4E0075F0A2C0E0C0F0120D031581158174C075F0A2C0E0C0F0747C75F05AC0E0C0F026
:203D6E00E53275F000C333C5F033C5F079737AAA12007889828A83E0A3F5F0E0C0F0C0E0DC
:203D8E00740375F000124AE37FFA12005074C075F0A2C0E0C0F0120D031581158174C0759D
:203DAE00F0A2C0E0C0F0749075F05AC0E0C0F0E53375F000C333C5F033C5F079737AAA12CE
:203DCE00007889828A83E0A3F5F0E0C0F0C0E0740375F000124AE37FFA12005074C075F01E
:203DEE00A2C0E0C0F0120D0315811581740A75F000C0E0C0F0120B9F1581158174C075F0C1
:203E0E00A2C0E0C0F074A475F05AC0E0C0F0E52275F000C0E0C0F0E523C0E0C0F0E51575F8
:203E2E00F000C0E0C0F0E514C0E0C0F0E51675F000C0E0C0F0E517C0E0C0F0740875F0000E
:203E4E00124AE37FF012005074C075F0A2C0E0C0F0120D0315811581E4F52EF5357F0102B8
:203E6E0001ED742C75F001C0E0C0F01246DB15811581227FFC7EFF1201EFE4F5F07F00121B
:203E8E0001D3F0A3C5F0F0C5F0E47F021201D3F07F021201D3E075F0007B107C00120181D1
:203EAE007012023F557F021201D3E0047F021201D3F080DCE47F031201D3F07F031201D33A
:203ECE00E075F0007B107C001201817012023F527F031201D3E0047F031201D3F080DC7F60
:203EEE00021201D3E075F0007B207C001200C0C0E0C0F07F031201D3E075F000C333C5F0F6
:203F0E0033C5F0D004D0032BC5F03CC5F079BB7AAC12007889828A83E0A3F5F0E0C5F045F5
:203F2E00F07003023F4F7F001201D3E0A3F5F0E0C5F012012D7F001201D3F0A3C5F0F0C57C
:203F4E00F0023EDE023EB37F001201D3E0A3F5F0E0C5F07F040201ED7FFD7EFF1201EFE49E
:203F6E007F001201D3F07F001201D3E075F0007B107C0012018170120241237F001201D34C
:203F8E00E0047F001201D3F080DC74017F021201D3F0E47F011201D3F07F011201D3E075BD
:203FAE00F0007B107C0012018170120241057F011201D3E0047F011201D3F080DC7F001211
:203FCE0001D3E075F0007B207C001200C0C0E0C0F07F011201D3E075F000C333C5F033C533
:203FEE00F0D004D0032BC5F03CC5F079BB7AAC12007889828A83E0A3F5F0E0C5F045F070AD
:20400E00030241027F021201D3E0700302406274C075F0A2C0E0C0F074E675F05AC0E0C0E8
:20402E00F07F001201D3E0244175F000C0E0C0F0740375F000124AE37FFA12005074C07584
:20404E00F0A2C0E0C0F0120D0315811581E47F021201D3F074C075F0A2C0E0C0F074EB7588
:20406E00F05AC0E0C0F07F011201D3E0240175F000C0E0C0F0740375F000124AE37FFA12D2
:20408E00005074C075F0A2C0E0C0F0120D03158115817F001201D3E075F0007B207C001216
:2040AE0000C0C0E0C0F07F011201D3E075F000C333C5F033C5F0D004D0032BC5F03CC5F02C
:2040CE0079BB7AAC12007889828A83E0A3F5F0E0C5F07B087C0012011BC0E0C0F012288D95
:2040EE0015811581742075F000C0E0C0F0120B9F15811581023FBC7F021201D3E0600302AC
:20410E004120740A75F000C0E0C0F0120B9F15811581023F897F030201ED7FFB7EFF1201CF
:20412E00EF90AEBBE0540475F0007B007C001201787F021201D3F078F9120044E60886F0E8
:20414E00904472020096740175F000C0E0C0F078F9120044E60886F0C0E0C0F0124CD1158A
:20416E008115811581158178FB120044F608A6F0181818E60886F0541FC5F05400C5F07B39
:20418E00087C0012010D0846C5F00846C5F07F001201D3F0A3C5F0F0C5F078F5120044E66C
:2041AE000886F07B207C001200C0C0E0C0F008E60886F0C333C5F033C5F0D004D0032BC5A4
:2041CE00F03CC5F079BB7AAC12007889828A83E0A3F5F0E0C5F045F0700302425578F51237
:2041EE000044E60886F07B207C001200C0C0E0C0F008E60886F0C333C5F033C5F0D004D02D
:20420E00032BC5F03CC5F079BB7AAC12007889828A83E0A3F5F0E0C5F07F001201D312004C
:20422E006A1201707003024241E47F021201D3F002425274EF75F05A7F031201D3F0A3C5D8
:20424E00F0F0C5F002426674F775F05A7F031201D3F0A3C5F0F0C5F078F5120044E608865B
:20426E00F07B207C001200C0C0E0C0F008E60886F0C333C5F033C5F0D004D0032BC5F03C45
:20428E00C5F079BB7AAC1200787F001201D3E0A3F5F0E0C5F089828A83F0A3C5F0F0C5F010
:2042AE0002448A78F5120044E60886F07B207C001200C0C0E0C0F008E60886F0C333C5F0A9
:2042CE0033C5F0D004D0032BC5F03CC5F079BB7AAC12007889828A83E0A3F5F0E0C5F04532
:2042EE00F0700302434778F5120044E60886F07B207C001200C0C0E0C0F008E60886F0C332
:20430E0033C5F033C5F0D004D0032BC5F03CC5F079BB7AAC120078E4F5F089828A83F0A3EF
:20432E00C5F0F0C5F074FB75F05A7F031201D3F0A3C5F0F0C5F002434EE47F021201D3F0C4
:20434E0002448AE4F5F078F7120044F608A6F078F7120044E60886F07B107C001201817029
:20436E001602445E78F7120044E60886F012012D18F608A6F080D878F5120044E60886F0E1
:20438E007B207C001200C0C0E0C0F008E60886F0C333C5F033C5F0D004D0032BC5F03CC54F
:2043AE00F079BB7AAC12007889828A83E0A3F5F0E0C5F045F0700302445B78F5120044E614
:2043CE000886F07B207C001200C0C0E0C0F008E60886F0C333C5F033C5F0D004D0032BC582
:2043EE00F03CC5F079BB7AAC120078E4F5F089828A83F0A3C5F0F0C5F07F021201D3E07065
:20440E000302445B74C075F0A2C0E0C0F0740375F05BC0E0C0F078F1120044E60886F02491
:20442E0041C5F03400C0F0C0E0740375F000124AE37FFA12005074C075F0A2C0E0C0F01261
:20444E000D0315811581E47F021201D3F0024372E47F021201D3F002448AE47F021201D3CA
:20446E00F002448A51431000B1421500B14214005441130054411200000068447F0212012C
:20448E00D3E0700302459A7F031201D3E0A3F5F0E0C0F0C0E0120D0315811581741975F0C7
:2044AE005BC0E0C0F0120D031581158178F5120044E60886F0C0E0C0F01227C81581158151
:2044CE00741F75F05BC0E0C0F0120D031581158178F7120044E60886F0C0E0C0F0122832F8
:2044EE0015811581742375F05BC0E0C0F0120D031581158178F9120044E60886F0C0E0C002
:20450E00F01228321581158174C075F0A2C0E0C0F0742775F05BC0E0C0F078F7120044E624
:20452E000886F0C0E0C0F0740375F000124AE37FFA12005074C075F0A2C0E0C0F0120D03FC
:20454E001581158178F7120044E60886F0C0E0C0F012288D15811581742075F000C0E0C05C
:20456E00F0120B9F1581158178F9120044E60886F0C0E0C0F012288D15811581743375F0DB
:20458E005BC0E0C0F0120D03158115817F050201ED78F9120044E60886F07B207C0012004C
:2045AE00C0C0E0C0F008E60886F0C333C5F033C5F0D004D0032BC5F03CC5F079BB7AAC12FA
:2045CE00007889828A83E0A3F5F0E0C5F045F070030246B090AEBBE0540475F0007B007C13
:2045EE0000120178700302467174C075F0A2C0E0C0F0743675F05BC0E0C0F0740275F000D6
:20460E00124AE3158115811581158174C075F0A2C0E0C0F0120D031581158178F912004455
:20462E00E60886F0C0E0C0F01227C815811581744175F05BC0E0C0F0120D03158115817800
:20464E00FB120044E60886F0C0E0C0F012283215811581740A75F000C0E0C0F0120B9F15AB
:20466E0081158178F9120044E60886F07B207C001200C0C0E0C0F008E60886F0C333C5F09A
:20468E0033C5F0D004D0032BC5F03CC5F079BB7AAC120078E4F5F089828A83F0A3C5F0F0AF
:2046AE00C5F02278FB120044E60886F090ACB5F0A3C5F0F0C5F0E4F5F090ACB7F0A3C5F006
:2046CE00F0C5F0E490ACBAF090ACB9F02278FB120044E60886F0C0E0C0F01246B115811525
:2046EE008174BB75F0ACC0E0C0F0E4C0E0C0E0E475F002C0E0C0F0124C0C7FFA02005F7F19
:20470E00FA7EFF1201EFE4F5F07F041201D3F0A3C5F0F0C5F090ACBAE00490ACBAF0540FD0
:20472E0090ACBAF0600302474690ACB9E00490ACB9F0540F90ACB9F07F041201D3E0A3F5AC
:20474E00F0E0C5F012012D7F041201D3F0A3C5F0F0C5F07B007C0112019760030247B090A2
:20476E00ACB9E075F0007B207C001200C0C0E0C0F090ACBAE075F000C333C5F033C5F0D0AA
:20478E0004D0032BC5F03CC5F079BB7AAC12007889828A83E0A3F5F0E0C5F045F0700302C0
:2047AE00472390ACB9E075F0007B207C001200C0C0E0C0F090ACBAE075F000C333C5F033F5
:2047CE00C5F0D004D0032BC5F03CC5F079BB7AAC12007889828A83E0A3F5F0E0C5F045F070
:2047EE0070030248D490ACB9E075F0007B207C001200C0C0E0C0F090ACBAE075F000C33376
:20480E00C5F033C5F0D004D0032BC5F03CC5F079BB7AAC12007889828A83E0A3F5F0E0C56C
:20482E00F05400C5F0541FC5F07B087C0012011B7F001201D3F0A3C5F0F0C5F090ACB9E0F5
:20484E0075F0007B207C001200C0C0E0C0F090ACBAE075F000C333C5F033C5F0D004D00337
:20486E002BC5F03CC5F079BB7AAC12007889828A83E0A3F5F0E0C5F054FFC5F05400C5F04F
:20488E007F021201D3F0A3C5F0F0C5F090ACB9E075F000C0E0C0F090ACBAE075F000C0E051
:2048AE00C0F07F001201D3E0A3F5F0E0C0F0C0E07F021201D3E0A3F5F0E0C0F0C0E01236F6
:2048CE00287FF81200507F060201ED7FFC7EFF1201EF90ACB7E0A3F5F0E0C5F012012D909A
:2048EE00ACB7F0A3C5F0F0C5F090ACB5E0A3F5F0E0C5F045F07003024990123E817F021285
:20490E0001D3F0A3C5F0F0C5F07F021201D3E0A3F5F0E0C5F045F0700302498D740175F00A
:20492E0000C0E0C0F090ACB5E0A3F5F0E0C5F07F021201D312006A1200DAC0E0C0F0124CAE
:20494E00D115811581158115817F001201D3F0A3C5F0F0C5F090ACB7E0A3F5F0E0C5F07F5F
:20496E00001201D312006A120197700302498D12470DE4F5F090ACB7F0A3C5F0F0C5F002C1
:20498E00499DE4F5F090ACB7F0A3C5F0F0C5F07F040201ED7FFC7EFF1201EF1201FA1223CB
:2049AE0004120207D2AF120898123E7090A38BE06003024A13744575F05BC0E0C0F0120D8F
:2049CE000315811581747175F05BC0E0C0F0120D0315811581747675F05BC0E0C0F0120D3E
:2049EE000315811581747C75F05BC0E0C0F0120D0315811581748275F05BC0E0C0F0120D07
:204A0E0003158115811212C4740175F00045F07003024AB7E4A21792E0F51F7003024A39D1
:204A2E00B297B297B297C2171248D91229167F021201D3F0A3C5F0F0C5F07BFF7CFF1201D4
:204A4E00787003024A8190ACB4E0540175F0007B017C001201707003024A7E7F021201D3E7
:204A6E00E0A3F5F0E0C0F0C0E0122AE615811581024A39120FD67F001201D3F0A3C5F0F029
:204A8E00C5F07B007C001201787003024AB47F001201D3E0A3F5F0E0C0F0C0E0121795158E
:204AAE008115811212C4024A1674AA75F05BC0E0C0F0120D03158115817F040201ED75F033
:204ACE0002A4041201452581F81201BB124E0E1201BB02046323F42581F8868208868308DF
:204AEE00024E0E0000000000000000002020202020000000000000000000000000000000AA
:204B0E00000000600101010101010101010101010101011818181818181818181801010125
:204B2E00010101010A0A0A0A0A0A02020202020202020202020202020202020202020101FD
:204B4E00010101010C0C0C0C0C0C04040404040404040404040404040404040404040101A9
:204B6E00010100C2D578FB120044E6904AF1C2E79355F060027401A2D575F00092F065F009
:204B8E0075F0002278FB120044E6A2E7B3E4F5F092E02275F00280CB75F00480C675F0066C
:204BAE0080C175F01680BC75F01780B775F05780B2D2D575F05780AD75F01080A675F008B6
:204BCE0080A175F001809C75F020809778FB120044E6C0E008E6C0E0124BA613D0F0D0E025
:204BEE00500224E02278FB120044E6C0E008E6C0E0124BA113D0F0D0E050E924202278F7C3
:204C0E00120044868208868308860708088603088604EB4C600AEFF0A31BBBFFF51C80F2DC
:204C2E002278FB1200448682088683E4FBFCFFE0A3B42D030FE0A3C39430B40A005012FAEE
:204C4E00740A75F0001200C02AFBE5F03400FC80E4EB8CF0DF030201452278F91200448603
:204C6E0082088683E0600DA380FA78F91200448682088683088601088602C9C582C9CAC5C2
:204C8E0083CAE0A3C9C582C9CAC583CAF06003A380E8E5828583F02278FB120044868208C9
:204CAE008683E4F5F0FAE06009A30ABA00F805F080F4EA2278FB120044E60886F030F73A6F
:204CCE0002014578F91200448603088604088605088606ED8EF012019D401CED8EF02278F9
:204CEE00F91200448603088604088605088606ED8EF012019D40E4EB8CF02278FB12004484
:204D0E00860308860485FEF0E5017F00120181600575F001E422EF0FF5F0A412018170F6AC
:204D2E00EF1475F0002278F91200448682088683088601088602C9C582C9CAC583CAE0F552
:204D4E00F0A3C9C582C9CAC583CAE0B5F0056009A380E37401500274FF02008B78F71200BC
:204D6E00448601080886F008088603088604EB4C600AA7F0091BBBFFF51C80F222124DE5AA
:204D8E00124DF1124DF8124DFFE0F7A30980F7124DE5124DF8124DF1124DFFE7F009A380BA
:204DAE00F7124DE5124DF1124DF8A882124DFFE6F7080980F7124DE5124DF1124DF8124DCC
:204DCE00FFE0A3CAC583CAC9C582C9F0A3CAC583CAC9C582C980E778FA12004486041886EF
:204DEE000318228683188682182286021886011822EB4C60061BBBFF011C221581158122A5
:204E0E00124F55868208868308E4FEFFE07006124F55E4F022B42551A3E0B42D054307806D
:204E2E00A3E0B4300343074024D0B40A00500BCE75F00AA42EFEA3E080EEE0B46413E6086C
:204E4E0086F030F708430720120145A6F018F68003B4750543070A8021B478054307108088
:204E6E0019B46F104307088011124F55F0A3124F55A38095B462624307027A00C004C00577
:204E8E00C006C007AB0753031F7C00E60886F01200DAA6F018F6EDD007D006D005D0042479
:204EAE0030B43A0040022407C0E00AE645F070CC124F55A902EF30E505742DF0A30A124F4F
:204ECE005ED0E0F0A3D9FA0808EF30E7A1EAC39E509C7420F0A30A80F4B4630DAA01124F8D
:204EEE0055124F5EE6F0A380DEB47331C082C08386820886837A00E06004A30A80F98683D6
:204F0E00188682124F55124F5E124F55E0A3124F556004F0A380F2D005D00480AAB4691B8B
:204F2E0086017A00E76004090A80F9124F55124F5E8601E76091F009A380F8F97A01124FCE
:204F4E0055124F5EE9809ECDC583CDCCC582CC22EE601A8FF020F715C002EAC39E500C7455
:204F6E002030F6027430F0A30A80EFD002224CFE4BFEB2F74CFE4BFEB2F74CFE4BFEA6F98D
:204F8E0024FE4CFE4BFEB2F74CFE4BFEB2F74CFE4BFE9AFB30F430F818FCE000000006906B
:204FAE000000060A9000000E0590000002099000000A0560000001096000000906600000BD
:204FCE00050A6000000D06A00000070AA000000F05A000000309A000000B05500000000927
:204FEE005000000806500000040A5000000C4D45434B4F4741494E46444C5048424A000003
:20500E000694000C000A94001C000594000400099400140005640002000964001200066480
:20502E00000A000A64001A0006A4000E000AA4001E0005A400060009A40016000554000081
:20504E0000095400100006540008000A540018000558000100056800030005980005000588
:20506E00A800070006580009000668000B000698000D0006A8000F00095800110009680048
:20508E001300099800150009A80017000A580019000A68001B000A98001D000AA8001F0CCD
:2050AE0010041102120A130E140615001608170D180519031A0B1B0F1C071D011E091F9E60
:2050CE0051A751B051B951C251CB51D451DD51E651EF51F95103520D52175221522B5235E9
:2050EE005243525152545258525C526352725280528D529E52AB52B852C652D352E1523059
:20510E00310030320030330030340030350030360030370030380030390031300031310061
:20512E00313200313300313400313500313600414600414E004F4E004F4600444D004252FB
:20514E00004C4600584300485200484100504400504400584400534E00534600535200004E
:20516E000102030405060708090A0B0C0D0E0F101112131415161718191A1B1C1D1E1FF041
:20518E0052F352F6525830310058313020007A5344657669636520310044657669636520B2
:2051AE003200446576696365203300446576696365203400446576696365203500446576A4
:2051CE00696365203600446576696365203700446576696365203800446576696365203942
:2051EE000044657669636520313000446576696365203131004465766963652031320044E7
:20520E00657669636520313300446576696365203134004465766963652031350044657626
:20522E0069636520313600416C6C20556E697473204F666600416C6C204C6967687473205D
:20524E004F6E004F6E004F66660044696D0042726967687400416C6C204C6967687473206D
:20526E004F666600457874656E64656420436F6465004861696C205265717565737400486A
:20528E0061696C2041636B6E6F776C65646765005072657365742044696D20300050726522
:2052AE007365742044696D203100457874656E646564204461746100537461747573206931
:2052CE0073204F6E00537461747573206973204F666600537461747573205265717565739C
:2052EE0074005858004F46004F4E00436F6E736F6C652073746174757320666C6167732066
:20530E00253032780A00205472616E733A20204865616420253032782C205461696C202528
:20532E003032782C2043747220253032782C204D617820253032780A00205265633A2020A2
:20534E0020204865616420253032782C205461696C20253032782C204374722025303278E5
:20536E002C204D617820253032780A00303132333435363738394142434445460030302062
:20538E000020002A2A2A2042616420636865636B73756D3A202532780A002A000A002A2115
:2053AE0020004F4B0A003E002A2A2A204E6F206164647265737320737472696E672E2E2E3B
:2053CE000A004E657420616464726573732069732025730A004E657420616464726573739D
:2053EE00205B25735D002E2020537461636B207573656420253032782F253032782E0A0075
:20540E004572726F7220666C61677320253032782E20204E6574776F726B20636865636BB2
:20542E0073756D206572726F72732025750A004C6F6767696E67206D6F64652069732025BB
:20544E00750A004E6574206D6F64652069732025750A002A2A2A204E20636D642073796E59
:20546E00746178206572726F720A002A2A2A20556E6B6E6F776E20636F6D6D616E643A2096
:20548E005B25735D0A004D616E75616C2072656D6F746520696E707574206D6F64652069FC
:2054AE00732025750A004661696C3D25752C0025750A002A2A2A205120636D642073796EC7
:2054CE00746178206572726F720A0052656672657368206379636C652025752073656320E9
:2054EE0077697468202575206D6F64756C65730A0045534554002A2A2A20556E6B6E6F77B4
:20550E006E20636F6D6D616E640A002A2A2A205220636D642073796E746178206572726F23
:20552E00720A002A2A2A205320636D642073796E746178206572726F720A00417661696C94
:20554E0061626C6520636F6D6D616E6473202876616C7565732061726520646563696D6184
:20556E006C20756E6C657373206E6F746564290A0020413D737472696E6720202B20207337
:20558E006574206E6574776F726B20616464726573730A0020442020202020202020202A3C
:2055AE00202064756D7020696E7465726E616C20737461747573207661726961626C6573CD
:2055CE0020286D6F737420696E20686578290A0020452020202020202020202A202064755B
:2055EE006D7020616E6420636C656172206572726F7220666C6167730A00204620202020DF
:20560E002020202020202020666C757368207472616E732F72656320627566666572730A92
:20562E0000204C206E20202020202020202020736574207265706F7274696E67206D6F647C
:20564E00657320286269746D6170706564290A00204D206E20202020202020202020736520
:20566E0074206D616E75616C2072656D6F746520636F6E74726F6C206D6F64650A00204E00
:20568E00206E202020202020202B2A20736574206E6574776F726B206D6F64650A00205064
:2056AE00202020202020202020202020646973706C617920616E6420636C65617220706FED
:2056CE00776572206661696C207374617475730A002051202020202020202020202020648F
:2056EE00756D7020616C6C206D6F64756C65730A0020512068202020202020202020206431
:20570E00756D7020616C6C206D6F64756C657320666F7220686F757365636F64650A002047
:20572E00512068206D6D2020202020202064756D702073696E676C65206D6F64756C65208A
:20574E00666F7220686F757365636F64650A00205120532020202020202020202064756DA1
:20576E007020616C6C206D6F64756C657320696E206865780A002052202020202020202061
:20578E002020202064756D70207265667265736820696E74657276616C0A002052206E2007
:2057AE00202020202020202020736574207265667265736820696E206D696E757465730A3A
:2057CE000020522043206E2020202020202020636C656172207265667265736820627566E5
:2057EE006665722C2073657420696E206D696E757465730A0020522053206E20202020208D
:20580E00202020736574207265667265736820696E207365636F6E64730A002052205120AC
:20582E0020202020202020202064756D702072656672657368207461626C6520656E747274
:20584E006965730A002052455345542020202020202020706572666F726D20706F77657204
:20586E002D6F6E20726573657420696E697469616C697A6174696F6E0A0020532068206D33
:20588E006D2063632072722073656E6420636F6D6D616E6420746F206D6F64756C652061B0
:2058AE007420686F757365636F64650A004D6F64756C6573206D757374206265207370656C
:2058CE0063696669656420776974682074776F206469676974733A202053204E203037207A
:2058EE004F4E0A002B206D61726B73206E6574776F726B2D6F6E6C7920636F6D6D616E6472
:20590E00730A002A206D61726B7320646562756767696E6720636F6D6D616E64730A002527
:20592E00633D253032780025303278002573005263763A2020483D0020442F463D0020289B
:20594E0000290A00253034780025633D002563253032753D25730A00456E513A2020483DDA
:20596E000020443D0020463D00205265703D252D3275202800290A00506F776572206C69DB
:20598E006E65207374617475733A0A00205472616E733A20204865616420253032782C209F
:2059AE005461696C20253032782C2043747220253032782C20004D617820253032782C20BF
:2059CE004F757450747220253034782C20457272466C61677320253032780A0020205B58AC
:2059EE004F7574486561645D202D3E20002025303278000A20205B584F75745461696C5DAC
:205A0E00202D3E20002025303278000A20205B584F75745074725D20202D3E2000202530A6
:205A2E003278000A2020584F7574426974735B5D202D3E2000202530327800205265633A4C
:205A4E00202020204865616420253032782C205461696C20253032782C2043747220253048
:205A6E0032782C204D617820253032780A0020205B58496E486561645D202D3E2025303426
:205A8E00780020205B58496E5461696C5D202D3E20253034780020506F7765726661696C7A
:205AAE003A2020414342697473202530327820253032782C2073746174652025752C206334
:205ACE0079632025752C20676F6F642025752C206261642025750A0025633A200025753D83
:205AEE0000436867205265660052656600436C722052656600436C7220416C6C2072656617
:205B0E0020666F7220483D25630A003A2020483D0020443D0020463D00205265703D252DC0
:205B2E003275202800290A0044656C2072656620483D0020443D000A504C2D4C696E6B20FC
:205B4E004E6574776F726B65642058313020436F6E74726F6C6C65722C2056657273696FA3
:205B6E006E2000312E32630020666F722000353020487A000A2020436F70797269676874C4
:205B8E00203139393220436972637569742043656C6C61722C20496E632E0A002D2D2D2057
:165BAE0046656C6C206F75742074686520626F74746F6D210A00A5
:00000001FF
